 j2gss

 Timestamp is ffffffff (Sun Feb  7 06:28:15 2106)

 Preferred load address is 10000000

 Start         Length     Name                   Class
 0001:00000000 000040faH .text$mn                CODE
 0002:00000000 0000009cH .idata$5                DATA
 0002:0000009c 00000004H .00cfg                  DATA
 0002:000000a0 00000004H .CRT$XCA                DATA
 0002:000000a4 00000004H .CRT$XCZ                DATA
 0002:000000a8 00000004H .CRT$XIA                DATA
 0002:000000ac 00000004H .CRT$XIZ                DATA
 0002:000000b0 00000004H .CRT$XPA                DATA
 0002:000000b4 00000004H .CRT$XPZ                DATA
 0002:000000b8 00000004H .CRT$XTA                DATA
 0002:000000bc 00000004H .CRT$XTZ                DATA
 0002:000000c0 00000000H .gfids$y                DATA
 0002:000000c0 00001db0H .rdata                  DATA
 0002:00001e70 00000004H .rdata$sxdata           DATA
 0002:00001e74 00000284H .rdata$zzzdbg           DATA
 0002:000020f8 00000004H .rtc$IAA                DATA
 0002:000020fc 00000004H .rtc$IZZ                DATA
 0002:00002100 00000004H .rtc$TAA                DATA
 0002:00002104 00000004H .rtc$TZZ                DATA
 0002:00002108 00000088H .xdata$x                DATA
 0002:00002190 00000820H .edata                  DATA
 0002:000029b0 00000064H .idata$2                DATA
 0002:00002a14 00000014H .idata$3                DATA
 0002:00002a28 0000009cH .idata$4                DATA
 0002:00002ac4 00000334H .idata$6                DATA
 0003:00000000 00000018H .data                   DATA
 0003:00000018 0000050cH .bss                    DATA
 0004:00000000 00000060H .rsrc$01                DATA
 0004:00000060 00000308H .rsrc$02                DATA

  Address         Publics by Value              Rva+Base       Lib:Object

 0000:00000000       ___guard_longjmp_count     00000000     <absolute>
 0000:00000000       ___dynamic_value_reloc_table 00000000     <absolute>
 0000:00000000       ___enclave_config          00000000     <absolute>
 0000:00000000       ___guard_iat_count         00000000     <absolute>
 0000:00000000       ___hybrid_code_map         00000000     <absolute>
 0000:00000000       ___hybrid_auxiliary_iat    00000000     <absolute>
 0000:00000000       ___guard_iat_table         00000000     <absolute>
 0000:00000000       ___hybrid_code_map_count   00000000     <absolute>
 0000:00000000       ___guard_fids_count        00000000     <absolute>
 0000:00000000       ___guard_fids_table        00000000     <absolute>
 0000:00000000       ___guard_longjmp_table     00000000     <absolute>
 0000:00000000       ___volatile_metadata       00000000     <absolute>
 0000:00000001       ___safe_se_handler_count   00000001     <absolute>
 0000:00000100       ___guard_flags             00000100     <absolute>
 0000:00000000       ___ImageBase               10000000     <linker-defined>
 0001:00000000       _Java_sun_security_jgss_wrapper_GSSLibStub_acceptContext@28 10001000 f   GSSLibStub.obj
 0001:00000565       _Java_sun_security_jgss_wrapper_GSSLibStub_acquireCred@24 10001565 f   GSSLibStub.obj
 0001:0000067e       _Java_sun_security_jgss_wrapper_GSSLibStub_canonicalizeName@16 1000167e f   GSSLibStub.obj
 0001:00000749       _Java_sun_security_jgss_wrapper_GSSLibStub_compareName@24 10001749 f   GSSLibStub.obj
 0001:000007c6       _Java_sun_security_jgss_wrapper_GSSLibStub_deleteContext@16 100017c6 f   GSSLibStub.obj
 0001:00000849       _Java_sun_security_jgss_wrapper_GSSLibStub_displayName@16 10001849 f   GSSLibStub.obj
 0001:00000989       _Java_sun_security_jgss_wrapper_GSSLibStub_exportContext@16 10001989 f   GSSLibStub.obj
 0001:00000a4b       _Java_sun_security_jgss_wrapper_GSSLibStub_exportName@16 10001a4b f   GSSLibStub.obj
 0001:00000ba3       _Java_sun_security_jgss_wrapper_GSSLibStub_getContextMech@16 10001ba3 f   GSSLibStub.obj
 0001:00000c2a       _Java_sun_security_jgss_wrapper_GSSLibStub_getContextName@20 10001c2a f   GSSLibStub.obj
 0001:00000cf0       _Java_sun_security_jgss_wrapper_GSSLibStub_getContextTime@16 10001cf0 f   GSSLibStub.obj
 0001:00000d87       _Java_sun_security_jgss_wrapper_GSSLibStub_getCredName@16 10001d87 f   GSSLibStub.obj
 0001:00000e1e       _Java_sun_security_jgss_wrapper_GSSLibStub_getCredTime@16 10001e1e f   GSSLibStub.obj
 0001:00000e8b       _Java_sun_security_jgss_wrapper_GSSLibStub_getCredUsage@16 10001e8b f   GSSLibStub.obj
 0001:00000ef0       _Java_sun_security_jgss_wrapper_GSSLibStub_getMechPtr@12 10001ef0 f   GSSLibStub.obj
 0001:00000fbe       _Java_sun_security_jgss_wrapper_GSSLibStub_getMic@24 10001fbe f   GSSLibStub.obj
 0001:000010a7       _Java_sun_security_jgss_wrapper_GSSLibStub_importContext@12 100020a7 f   GSSLibStub.obj
 0001:00001236       _Java_sun_security_jgss_wrapper_GSSLibStub_importName@16 10002236 f   GSSLibStub.obj
 0001:00001355       _Java_sun_security_jgss_wrapper_GSSLibStub_indicateMechs@8 10002355 f   GSSLibStub.obj
 0001:00001373       _Java_sun_security_jgss_wrapper_GSSLibStub_init@16 10002373 f   GSSLibStub.obj
 0001:00001493       _Java_sun_security_jgss_wrapper_GSSLibStub_initContext@36 10002493 f   GSSLibStub.obj
 0001:000017b3       _Java_sun_security_jgss_wrapper_GSSLibStub_inquireContext@16 100027b3 f   GSSLibStub.obj
 0001:00001958       _Java_sun_security_jgss_wrapper_GSSLibStub_inquireNamesForMech@8 10002958 f   GSSLibStub.obj
 0001:000019e8       _Java_sun_security_jgss_wrapper_GSSLibStub_releaseCred@16 100029e8 f   GSSLibStub.obj
 0001:00001a69       _Java_sun_security_jgss_wrapper_GSSLibStub_releaseName@16 10002a69 f   GSSLibStub.obj
 0001:00001ad0       _Java_sun_security_jgss_wrapper_GSSLibStub_unwrap@24 10002ad0 f   GSSLibStub.obj
 0001:00001c49       _Java_sun_security_jgss_wrapper_GSSLibStub_verifyMic@28 10002c49 f   GSSLibStub.obj
 0001:00001dba       _Java_sun_security_jgss_wrapper_GSSLibStub_wrap@24 10002dba f   GSSLibStub.obj
 0001:00001f2a       _Java_sun_security_jgss_wrapper_GSSLibStub_wrapSizeLimit@28 10002f2a f   GSSLibStub.obj
 0001:00001fca       ___local_stdio_printf_options 10002fca f i GSSLibStub.obj
 0001:00001fd0       __vfprintf_l               10002fd0 f i GSSLibStub.obj
 0001:00001ff4       _deleteGSSCB               10002ff4 f   GSSLibStub.obj
 0001:00002045       _inquireCred               10003045 f   GSSLibStub.obj
 0001:000020f9       _newGSSCB                  100030f9 f   GSSLibStub.obj
 0001:0000229b       _printf                    1000329b f i GSSLibStub.obj
 0001:000022b9       _setSupplementaryInfo      100032b9 f   GSSLibStub.obj
 0001:00002325       _loadNative                10003325 f   NativeFunc.obj
 0001:000026f3       _JNI_OnLoad@8              100036f3 f   NativeUtil.obj
 0001:00002dca       _JNI_OnUnload@8            10003dca f   NativeUtil.obj
 0001:00002e50       _checkStatus               10003e50 f   NativeUtil.obj
 0001:00002f76       _deleteGSSOID              10003f76 f   NativeUtil.obj
 0001:00002f93       _deleteGSSOIDSet           10003f93 f   NativeUtil.obj
 0001:00002fb7       _getGSSTime                10003fb7 f   NativeUtil.obj
 0001:00002fc8       _getJavaBuffer             10003fc8 f   NativeUtil.obj
 0001:0000302a       _getJavaErrorCode          1000402a f   NativeUtil.obj
 0001:0000306b       _getJavaOID                1000406b f   NativeUtil.obj
 0001:0000311b       _getJavaOIDArray           1000411b f   NativeUtil.obj
 0001:000031b6       _getJavaString             100041b6 f   NativeUtil.obj
 0001:00003239       _getJavaTime               10004239 f   NativeUtil.obj
 0001:00003256       _getMinorMessage           10004256 f   NativeUtil.obj
 0001:000032a6       _initGSSBuffer             100042a6 f   NativeUtil.obj
 0001:0000331d       _newGSSOID                 1000431d f   NativeUtil.obj
 0001:000033d0       _newGSSOIDSet              100043d0 f   NativeUtil.obj
 0001:00003426       _resetGSSBuffer            10004426 f   NativeUtil.obj
 0001:00003442       _sameMech                  10004442 f   NativeUtil.obj
 0001:00003469       _throwByName               10004469 f   NativeUtil.obj
 0001:00003489       _throwOutOfMemoryError     10004489 f   NativeUtil.obj
 0001:0000349f       @__security_check_cookie@4 1000449f f   MSVCRT:secchk.obj
 0001:000037d0       __DllMainCRTStartup@12     100047d0 f   MSVCRT:dll_dllmain.obj
 0001:000037f3       ___raise_securityfailure   100047f3 f   MSVCRT:gs_report.obj
 0001:0000381b       ___report_gsfailure        1000481b f   MSVCRT:gs_report.obj
 0001:00003961       ___security_init_cookie    10004961 f   MSVCRT:gs_support.obj
 0001:000039ac       _DllMain@12                100049ac f   MSVCRT:dll_dllmain_stub.obj
 0001:000039ce       ?__scrt_initialize_type_info@@YAXXZ 100049ce f   MSVCRT:tncleanup.obj
 0001:000039da       ?__scrt_uninitialize_type_info@@YAXXZ 100049da f   MSVCRT:tncleanup.obj
 0001:000039e6       ___local_stdio_scanf_options 100049e6 f i MSVCRT:default_local_stdio_options.obj
 0001:000039ec       ___scrt_initialize_default_local_stdio_options 100049ec f   MSVCRT:default_local_stdio_options.obj
 0001:00003a4d       ___scrt_acquire_startup_lock 10004a4d f   MSVCRT:utility.obj
 0001:00003a7f       ___scrt_dllmain_after_initialize_c 10004a7f f   MSVCRT:utility.obj
 0001:00003aaa       ___scrt_dllmain_before_initialize_c 10004aaa f   MSVCRT:utility.obj
 0001:00003ab8       ___scrt_dllmain_crt_thread_attach 10004ab8 f   MSVCRT:utility.obj
 0001:00003ad7       ___scrt_dllmain_crt_thread_detach 10004ad7 f   MSVCRT:utility.obj
 0001:00003ae4       ___scrt_dllmain_exception_filter 10004ae4 f   MSVCRT:utility.obj
 0001:00003b18       ___scrt_dllmain_uninitialize_c 10004b18 f   MSVCRT:utility.obj
 0001:00003b3b       ___scrt_dllmain_uninitialize_critical 10004b3b f   MSVCRT:utility.obj
 0001:00003b48       ___scrt_initialize_crt     10004b48 f   MSVCRT:utility.obj
 0001:00003b81       ___scrt_initialize_onexit_tables 10004b81 f   MSVCRT:utility.obj
 0001:00003c26       ___scrt_is_nonwritable_in_current_image 10004c26 f   MSVCRT:utility.obj
 0001:00003cba       ___scrt_release_startup_lock 10004cba f   MSVCRT:utility.obj
 0001:00003cd7       ___scrt_uninitialize_crt   10004cd7 f   MSVCRT:utility.obj
 0001:00003cff       ___scrt_get_dyn_tls_init_callback 10004cff f   MSVCRT:dyn_tls_init.obj
 0001:00003d05       ___scrt_fastfail           10004d05 f   MSVCRT:utility_desktop.obj
 0001:00003e1f       __crt_debugger_hook        10004e1f f   MSVCRT:utility_desktop.obj
 0001:00003e27       __RTC_Initialize           10004e27 f   MSVCRT:initsect.obj
 0001:00003e53       __RTC_Terminate            10004e53 f   MSVCRT:initsect.obj
 0001:00003e80       __SEH_prolog4              10004e80 f   MSVCRT:sehprolg4.obj
 0001:00003ec6       __SEH_epilog4              10004ec6 f   MSVCRT:sehprolg4.obj
 0001:00003edb       __except_handler4          10004edb f   MSVCRT:chandler4gs.obj
 0001:00003efe       @_guard_check_icall_nop@4  10004efe f i MSVCRT:guard_support.obj
 0001:00003eff       ___isa_available_init      10004eff f   MSVCRT:cpu_disp.obj
 0001:00004096       __get_startup_argv_mode    10005096 f   MSVCRT:argv_mode.obj
 0001:0000409a       ___scrt_is_ucrt_dll_in_use 1000509a f   MSVCRT:ucrt_detection.obj
 0001:000040a6       _IsProcessorFeaturePresent@4 100050a6 f   kernel32:KERNEL32.dll
 0001:000040ac       _memcmp                    100050ac f   vcruntime:VCRUNTIME140.dll
 0001:000040b2       _memset                    100050b2 f   vcruntime:VCRUNTIME140.dll
 0001:000040b8       ___std_type_info_destroy_list 100050b8 f   vcruntime:VCRUNTIME140.dll
 0001:000040be       __except_handler4_common   100050be f   vcruntime:VCRUNTIME140.dll
 0001:000040c4       __initterm                 100050c4 f   ucrt:api-ms-win-crt-runtime-l1-1-0.dll
 0001:000040ca       __initterm_e               100050ca f   ucrt:api-ms-win-crt-runtime-l1-1-0.dll
 0001:000040d0       __seh_filter_dll           100050d0 f   ucrt:api-ms-win-crt-runtime-l1-1-0.dll
 0001:000040d6       __configure_narrow_argv    100050d6 f   ucrt:api-ms-win-crt-runtime-l1-1-0.dll
 0001:000040dc       __initialize_narrow_environment 100050dc f   ucrt:api-ms-win-crt-runtime-l1-1-0.dll
 0001:000040e2       __initialize_onexit_table  100050e2 f   ucrt:api-ms-win-crt-runtime-l1-1-0.dll
 0001:000040e8       __execute_onexit_table     100050e8 f   ucrt:api-ms-win-crt-runtime-l1-1-0.dll
 0001:000040ee       __cexit                    100050ee f   ucrt:api-ms-win-crt-runtime-l1-1-0.dll
 0001:000040f4       ___acrt_uninitialize       100050f4 f   MSVCRT:ucrt_stubs.obj
 0001:000040f4       ___vcrt_initialize         100050f4 f   MSVCRT:ucrt_stubs.obj
 0001:000040f4       ___acrt_thread_attach      100050f4 f   MSVCRT:ucrt_stubs.obj
 0001:000040f4       ___scrt_stub_for_acrt_thread_detach 100050f4 f   MSVCRT:ucrt_stubs.obj
 0001:000040f4       ___vcrt_thread_attach      100050f4 f   MSVCRT:ucrt_stubs.obj
 0001:000040f4       ___acrt_thread_detach      100050f4 f   MSVCRT:ucrt_stubs.obj
 0001:000040f4       ___vcrt_uninitialize       100050f4 f   MSVCRT:ucrt_stubs.obj
 0001:000040f4       ___scrt_stub_for_acrt_uninitialize 100050f4 f   MSVCRT:ucrt_stubs.obj
 0001:000040f4       ___vcrt_thread_detach      100050f4 f   MSVCRT:ucrt_stubs.obj
 0001:000040f4       ___acrt_uninitialize_critical 100050f4 f   MSVCRT:ucrt_stubs.obj
 0001:000040f4       ___scrt_stub_for_acrt_initialize 100050f4 f   MSVCRT:ucrt_stubs.obj
 0001:000040f4       ___vcrt_uninitialize_critical 100050f4 f   MSVCRT:ucrt_stubs.obj
 0001:000040f4       ___acrt_initialize         100050f4 f   MSVCRT:ucrt_stubs.obj
 0001:000040f4       ___scrt_stub_for_acrt_thread_attach 100050f4 f   MSVCRT:ucrt_stubs.obj
 0001:000040f4       ___scrt_stub_for_acrt_uninitialize_critical 100050f4 f   MSVCRT:ucrt_stubs.obj
 0001:000040f7       ___scrt_stub_for_is_c_termination_complete 100050f7 f   MSVCRT:ucrt_stubs.obj
 0001:000040f7       __is_c_termination_complete 100050f7 f   MSVCRT:ucrt_stubs.obj
 0002:00000000       __imp__GetLastError@0      10006000     kernel32:KERNEL32.dll
 0002:00000004       __imp__FormatMessageA@28   10006004     kernel32:KERNEL32.dll
 0002:00000008       __imp__CloseHandle@4       10006008     kernel32:KERNEL32.dll
 0002:0000000c       __imp__GetProcAddress@8    1000600c     kernel32:KERNEL32.dll
 0002:00000010       __imp__LoadLibraryA@4      10006010     kernel32:KERNEL32.dll
 0002:00000014       __imp__UnhandledExceptionFilter@4 10006014     kernel32:KERNEL32.dll
 0002:00000018       __imp__SetUnhandledExceptionFilter@4 10006018     kernel32:KERNEL32.dll
 0002:0000001c       __imp__GetCurrentProcess@0 1000601c     kernel32:KERNEL32.dll
 0002:00000020       __imp__TerminateProcess@8  10006020     kernel32:KERNEL32.dll
 0002:00000024       __imp__IsProcessorFeaturePresent@4 10006024     kernel32:KERNEL32.dll
 0002:00000028       __imp__QueryPerformanceCounter@4 10006028     kernel32:KERNEL32.dll
 0002:0000002c       __imp__GetCurrentProcessId@0 1000602c     kernel32:KERNEL32.dll
 0002:00000030       __imp__GetCurrentThreadId@0 10006030     kernel32:KERNEL32.dll
 0002:00000034       __imp__GetSystemTimeAsFileTime@4 10006034     kernel32:KERNEL32.dll
 0002:00000038       __imp__DisableThreadLibraryCalls@4 10006038     kernel32:KERNEL32.dll
 0002:0000003c       __imp__InitializeSListHead@4 1000603c     kernel32:KERNEL32.dll
 0002:00000040       __imp__IsDebuggerPresent@0 10006040     kernel32:KERNEL32.dll
 0002:00000044       \177KERNEL32_NULL_THUNK_DATA 10006044     kernel32:KERNEL32.dll
 0002:00000048       __imp__memcmp              10006048     vcruntime:VCRUNTIME140.dll
 0002:0000004c       __imp__memset              1000604c     vcruntime:VCRUNTIME140.dll
 0002:00000050       __imp____std_type_info_destroy_list 10006050     vcruntime:VCRUNTIME140.dll
 0002:00000054       __imp___except_handler4_common 10006054     vcruntime:VCRUNTIME140.dll
 0002:00000058       \177VCRUNTIME140_NULL_THUNK_DATA 10006058     vcruntime:VCRUNTIME140.dll
 0002:0000005c       __imp__malloc              1000605c     ucrt:api-ms-win-crt-heap-l1-1-0.dll
 0002:00000060       __imp__free                10006060     ucrt:api-ms-win-crt-heap-l1-1-0.dll
 0002:00000064       \177api-ms-win-crt-heap-l1-1-0_NULL_THUNK_DATA 10006064     ucrt:api-ms-win-crt-heap-l1-1-0.dll
 0002:00000068       __imp___cexit              10006068     ucrt:api-ms-win-crt-runtime-l1-1-0.dll
 0002:0000006c       __imp___initterm           1000606c     ucrt:api-ms-win-crt-runtime-l1-1-0.dll
 0002:00000070       __imp___initterm_e         10006070     ucrt:api-ms-win-crt-runtime-l1-1-0.dll
 0002:00000074       __imp___seh_filter_dll     10006074     ucrt:api-ms-win-crt-runtime-l1-1-0.dll
 0002:00000078       __imp___configure_narrow_argv 10006078     ucrt:api-ms-win-crt-runtime-l1-1-0.dll
 0002:0000007c       __imp___initialize_narrow_environment 1000607c     ucrt:api-ms-win-crt-runtime-l1-1-0.dll
 0002:00000080       __imp___initialize_onexit_table 10006080     ucrt:api-ms-win-crt-runtime-l1-1-0.dll
 0002:00000084       __imp___execute_onexit_table 10006084     ucrt:api-ms-win-crt-runtime-l1-1-0.dll
 0002:00000088       \177api-ms-win-crt-runtime-l1-1-0_NULL_THUNK_DATA 10006088     ucrt:api-ms-win-crt-runtime-l1-1-0.dll
 0002:0000008c       __imp__fflush              1000608c     ucrt:api-ms-win-crt-stdio-l1-1-0.dll
 0002:00000090       __imp____acrt_iob_func     10006090     ucrt:api-ms-win-crt-stdio-l1-1-0.dll
 0002:00000094       __imp____stdio_common_vfprintf 10006094     ucrt:api-ms-win-crt-stdio-l1-1-0.dll
 0002:00000098       \177api-ms-win-crt-stdio-l1-1-0_NULL_THUNK_DATA 10006098     ucrt:api-ms-win-crt-stdio-l1-1-0.dll
 0002:0000009c       ___guard_check_icall_fptr  1000609c     MSVCRT:guard_support.obj
 0002:000000a0       ___xc_a                    100060a0     MSVCRT:initializers.obj
 0002:000000a4       ___xc_z                    100060a4     MSVCRT:initializers.obj
 0002:000000a8       ___xi_a                    100060a8     MSVCRT:initializers.obj
 0002:000000ac       ___xi_z                    100060ac     MSVCRT:initializers.obj
 0002:000000b0       ___xp_a                    100060b0     MSVCRT:initializers.obj
 0002:000000b4       ___xp_z                    100060b4     MSVCRT:initializers.obj
 0002:000000b8       ___xt_a                    100060b8     MSVCRT:initializers.obj
 0002:000000bc       ___xt_z                    100060bc     MSVCRT:initializers.obj
 0002:000000c0       _TYPE_CRED_NAME            100060c0     GSSLibStub.obj
 0002:000000c4       _TYPE_CRED_TIME            100060c4     GSSLibStub.obj
 0002:000000c8       _TYPE_CRED_USAGE           100060c8     GSSLibStub.obj
 0002:000000cc       ??_C@_0CH@IFIMLFDG@?$FLGSSLibStub_init?$FN?5GSS?5lib?5name?5@ 100060cc     GSSLibStub.obj
 0002:000000f4       ??_C@_0BE@FBKICJJF@?$FLGSSLibStub?3?$CFd?$FN?5?$CFs?6@ 100060f4     GSSLibStub.obj
 0002:00000108       ??_C@_0CO@DHBKBJOL@?$FLGSSLibStub?3?$CFd?$FN?5?$FLGSSLibStub_ini@ 10006108     GSSLibStub.obj
 0002:00000138       ??_C@_0DG@BBGFBBEA@sun?1security?1jgss?1krb5?1internal@ 10006138     GSSLibStub.obj
 0002:00000170       ??_C@_0BN@LGLCDLKI@GSS?9API?3?5Unknown?5failure?5?$CFd?6@ 10006170     GSSLibStub.obj
 0002:00000190       ??_C@_0N@DCKHCLFP@GSS?9API?3?5?$CFs?6@ 10006190     GSSLibStub.obj
 0002:000001a0       ??_C@_0BI@FIIPHNCE@?$FLGSSLibStub_getMechPtr?$FN@ 100061a0     GSSLibStub.obj
 0002:000001b8       ??_C@_0CB@EEKJDBHK@?$FLGSSLibStub_inquireNamesForMech@ 100061b8     GSSLibStub.obj
 0002:000001dc       ??_C@_0CO@FNFLNOMG@?$FLGSSLibStub?3?$CFd?$FN?5?$FLGSSLibStub_rel@ 100061dc     GSSLibStub.obj
 0002:0000020c       ??_C@_0BJ@CBIHLCMJ@?$FLGSSLibStub_releaseName?$FN@ 1000620c     GSSLibStub.obj
 0002:00000228       ??_C@_0BI@DFKAFKP@?$FLGSSLibStub_importName?$FN@ 10006228     GSSLibStub.obj
 0002:00000240       ??_C@_0CM@NEMNNPAK@?$FLGSSLibStub?3?$CFd?$FN?5?$FLGSSLibStub_imp@ 10006240     GSSLibStub.obj
 0002:0000026c       ??_C@_0DC@EDJDCFOA@?$FLGSSLibStub?3?$CFd?$FN?5?$FLGSSLibStub_com@ 1000626c     GSSLibStub.obj
 0002:000002a0       ??_C@_0BJ@GOICLAAF@?$FLGSSLibStub_compareName?$FN@ 100062a0     GSSLibStub.obj
 0002:000002bc       ??_C@_0DD@PNOHLKNJ@?$FLGSSLibStub?3?$CFd?$FN?5?$FLGSSLibStub_can@ 100062bc     GSSLibStub.obj
 0002:000002f0       ??_C@_0DF@OMPECPHP@?$FLGSSLibStub?3?$CFd?$FN?5?$FLGSSLibStub_can@ 100062f0     GSSLibStub.obj
 0002:00000328       ??_C@_0BO@MEBIAJAG@?$FLGSSLibStub_canonicalizeName?$FN@ 10006328     GSSLibStub.obj
 0002:00000348       ??_C@_0CN@HMNALJKN@?$FLGSSLibStub?3?$CFd?$FN?5?$FLGSSLibStub_exp@ 10006348     GSSLibStub.obj
 0002:00000378       ??_C@_0DA@BMLGEALK@?$FLGSSLibStub_exportName?$FN?5canonic@ 10006378     GSSLibStub.obj
 0002:000003a8       ??_C@_0BI@NJPBCAKH@?$FLGSSLibStub_exportName?$FN@ 100063a8     GSSLibStub.obj
 0002:000003c0       ??_C@_0CO@JNAHONNN@?$FLGSSLibStub?3?$CFd?$FN?5?$FLGSSLibStub_dis@ 100063c0     GSSLibStub.obj
 0002:000003f0       ??_C@_0BJ@KDEJNLFF@?$FLGSSLibStub_displayName?$FN@ 100063f0     GSSLibStub.obj
 0002:0000040c       ??_C@_0BJ@KNGBMLML@?$FLGSSLibStub_acquireCred?$FN@ 1000640c     GSSLibStub.obj
 0002:00000428       ??_C@_0DO@GCCNNHHE@?$FLGSSLibStub?3?$CFd?$FN?5?$FLGSSLibStub_acq@ 10006428     GSSLibStub.obj
 0002:00000468       ??_C@_0DD@KNGMBANC@?$FLGSSLibStub?3?$CFd?$FN?5?$FLGSSLibStub_acq@ 10006468     GSSLibStub.obj
 0002:0000049c       ??_C@_0CO@CNCEALKM@?$FLGSSLibStub?3?$CFd?$FN?5?$FLGSSLibStub_rel@ 1000649c     GSSLibStub.obj
 0002:000004cc       ??_C@_0BJ@HOCPAOJN@?$FLGSSLibStub_releaseCred?$FN@ 100064cc     GSSLibStub.obj
 0002:000004e8       ??_C@_0CH@HAGGPEEB@?$FLGSSLibStub?3?$CFd?$FN?5?$FLgss_inquire_cr@ 100064e8     GSSLibStub.obj
 0002:00000510       ??_C@_0BD@NFEKOCFD@?$FLgss_inquire_cred?$FN@ 10006510     GSSLibStub.obj
 0002:00000524       ??_C@_0CO@DNJNIEFL@?$FLGSSLibStub?3?$CFd?$FN?5?$FLGSSLibStub_get@ 10006524     GSSLibStub.obj
 0002:00000554       ??_C@_0DD@HJKBNIGO@?$FLGSSLibStub?3?$CFd?$FN?5?$FLGSSLibStub_get@ 10006554     GSSLibStub.obj
 0002:00000588       ??_C@_0CO@GCBDFIOA@?$FLGSSLibStub?3?$CFd?$FN?5?$FLGSSLibStub_get@ 10006588     GSSLibStub.obj
 0002:000005b8       ??_C@_0CP@OAPFJNOP@?$FLGSSLibStub?3?$CFd?$FN?5?$FLGSSLibStub_get@ 100065b8     GSSLibStub.obj
 0002:000005e8       ??_C@_0BL@FKHNPAJG@?$FLGSSLibStub_importContext?$FN@ 100065e8     GSSLibStub.obj
 0002:00000604       ??_C@_0DI@ODFIHJGC@?$FLGSSLibStub?3?$CFd?$FN?5?$FLGSSLibStub_imp@ 10006604     GSSLibStub.obj
 0002:0000063c       ??_C@_0CD@BCECEGFB@?$FLGSSLibStub_importContext?$FN?5getM@ 1000663c     GSSLibStub.obj
 0002:00000660       ??_C@_0CD@ICJKNONJ@?$FLGSSLibStub_importContext?$FN?5clea@ 10006660     GSSLibStub.obj
 0002:00000684       ??_C@_0BJ@BFLGHPHA@?$FLGSSLibStub_initContext?$FN@ 10006684     GSSLibStub.obj
 0002:000006a0       ??_C@_0EI@DLLKPAO@?$FLGSSLibStub?3?$CFd?$FN?5?$FLGSSLibStub_ini@ 100066a0     GSSLibStub.obj
 0002:000006e8       ??_C@_0EP@BOGHBFMJ@?$FLGSSLibStub?3?$CFd?$FN?5?$FLGSSLibStub_ini@ 100066e8     GSSLibStub.obj
 0002:00000738       ??_C@_0DK@PIOENCNN@?$FLGSSLibStub?3?$CFd?$FN?5?$FLGSSLibStub_ini@ 10006738     GSSLibStub.obj
 0002:00000774       ??_C@_0DJ@EHOIIEEF@?$FLGSSLibStub?3?$CFd?$FN?5?$FLGSSLibStub_ini@ 10006774     GSSLibStub.obj
 0002:000007b0       ??_C@_0CN@EFAHJDCF@?$FLGSSLibStub_initContext?$FN?5contex@ 100067b0     GSSLibStub.obj
 0002:000007e0       ??_C@_0DB@LEECDODG@?$FLGSSLibStub_initContext?$FN?5contex@ 100067e0     GSSLibStub.obj
 0002:00000814       ??_C@_0BL@OFPJPCCF@?$FLGSSLibStub_acceptContext?$FN@ 10006814     GSSLibStub.obj
 0002:00000830       ??_C@_0EK@GNNFCOCF@?$FLGSSLibStub?3?$CFd?$FN?5?$FLGSSLibStub_acc@ 10006830     GSSLibStub.obj
 0002:00000880       ??_C@_0FI@PEIDNCN@?$FLGSSLibStub?3?$CFd?$FN?5?$FLGSSLibStub_acc@ 10006880     GSSLibStub.obj
 0002:000008d8       ??_C@_0DM@IGEPIBMJ@?$FLGSSLibStub?3?$CFd?$FN?5?$FLGSSLibStub_acc@ 100068d8     GSSLibStub.obj
 0002:00000914       ??_C@_0DL@FNMHCNEI@?$FLGSSLibStub?3?$CFd?$FN?5?$FLGSSLibStub_acc@ 10006914     GSSLibStub.obj
 0002:00000950       ??_C@_0CD@POJPGDLJ@?$FLGSSLibStub_acceptContext?$FN?5inqu@ 10006950     GSSLibStub.obj
 0002:00000974       ??_C@_0DO@JCJNAGBN@?$FLGSSLibStub?3?$CFd?$FN?5?$FLGSSLibStub_acc@ 10006974     GSSLibStub.obj
 0002:000009b4       ??_C@_0DL@MGJILOGD@?$FLGSSLibStub?3?$CFd?$FN?5?$FLGSSLibStub_acc@ 100069b4     GSSLibStub.obj
 0002:000009f0       ??_C@_0CP@IEEDNBPF@?$FLGSSLibStub_acceptContext?$FN?5cont@ 100069f0     GSSLibStub.obj
 0002:00000a20       ??_C@_0EB@KEOJNLHA@?$FLGSSLibStub?3?$CFd?$FN?5?$FLGSSLibStub_acc@ 10006a20     GSSLibStub.obj
 0002:00000a64       ??_C@_0DD@JJHOKGCG@?$FLGSSLibStub_acceptContext?$FN?5cont@ 10006a64     GSSLibStub.obj
 0002:00000a98       ??_C@_0DA@NPPDLHMN@?$FLGSSLibStub?3?$CFd?$FN?5?$FLGSSLibStub_inq@ 10006a98     GSSLibStub.obj
 0002:00000ac8       ??_C@_0EH@KBCPMKIM@?$FLGSSLibStub?3?$CFd?$FN?5?$FLGSSLibStub_inq@ 10006ac8     GSSLibStub.obj
 0002:00000b10       ??_C@_0BM@IFAECBDO@?$FLGSSLibStub_inquireContext?$FN@ 10006b10     GSSLibStub.obj
 0002:00000b2c       ??_C@_0DB@IFOABMAJ@?$FLGSSLibStub?3?$CFd?$FN?5?$FLGSSLibStub_get@ 10006b2c     GSSLibStub.obj
 0002:00000b60       ??_C@_0BM@COJKOILK@?$FLGSSLibStub_getContextMech?$FN@ 10006b60     GSSLibStub.obj
 0002:00000b7c       ??_C@_0DK@FHHIMKKL@?$FLGSSLibStub?3?$CFd?$FN?5?$FLGSSLibStub_get@ 10006b7c     GSSLibStub.obj
 0002:00000bb8       ??_C@_0BP@DPDPDKIA@?$FLGSSLibStub_inquireContextAll?$FN@ 10006bb8     GSSLibStub.obj
 0002:00000bd8       ??_C@_0DG@BMLALGFC@?$FLGSSLibStub?3?$CFd?$FN?5?$FLGSSLibStub_get@ 10006bd8     GSSLibStub.obj
 0002:00000c10       ??_C@_0DA@MEKCMMFO@?$FLGSSLibStub?3?$CFd?$FN?5?$FLGSSLibStub_get@ 10006c10     GSSLibStub.obj
 0002:00000c40       ??_C@_0BM@CHLELCII@?$FLGSSLibStub_getContextTime?$FN@ 10006c40     GSSLibStub.obj
 0002:00000c5c       ??_C@_0CP@FHIJGEMK@?$FLGSSLibStub?3?$CFd?$FN?5?$FLGSSLibStub_del@ 10006c5c     GSSLibStub.obj
 0002:00000c8c       ??_C@_0BL@HBHJELHJ@?$FLGSSLibStub_deleteContext?$FN@ 10006c8c     GSSLibStub.obj
 0002:00000ca8       ??_C@_0CP@PCFDMPGD@?$FLGSSLibStub?3?$CFd?$FN?5?$FLGSSLibStub_wra@ 10006ca8     GSSLibStub.obj
 0002:00000cd8       ??_C@_0BL@GNPIIACB@?$FLGSSLibStub_wrapSizeLimit?$FN@ 10006cd8     GSSLibStub.obj
 0002:00000cf4       ??_C@_0CP@PCNODFIJ@?$FLGSSLibStub?3?$CFd?$FN?5?$FLGSSLibStub_exp@ 10006cf4     GSSLibStub.obj
 0002:00000d24       ??_C@_0BL@PNJJALHD@?$FLGSSLibStub_exportContext?$FN@ 10006d24     GSSLibStub.obj
 0002:00000d40       ??_C@_0CI@PNJGMJEH@?$FLGSSLibStub?3?$CFd?$FN?5?$FLGSSLibStub_get@ 10006d40     GSSLibStub.obj
 0002:00000d68       ??_C@_0BE@PDIMELDO@?$FLGSSLibStub_getMic?$FN@ 10006d68     GSSLibStub.obj
 0002:00000d7c       ??_C@_0CL@HBMACJOD@?$FLGSSLibStub?3?$CFd?$FN?5?$FLGSSLibStub_ver@ 10006d7c     GSSLibStub.obj
 0002:00000da8       ??_C@_0BH@IPGHLHPO@?$FLGSSLibStub_verifyMic?$FN@ 10006da8     GSSLibStub.obj
 0002:00000dc0       ??_C@_0CG@IAFPKAEF@?$FLGSSLibStub?3?$CFd?$FN?5?$FLGSSLibStub_wra@ 10006dc0     GSSLibStub.obj
 0002:00000de8       ??_C@_0BC@HKCNLDAH@?$FLGSSLibStub_wrap?$FN@ 10006de8     GSSLibStub.obj
 0002:00000dfc       ??_C@_0CI@KBPIBEIG@?$FLGSSLibStub?3?$CFd?$FN?5?$FLGSSLibStub_unw@ 10006dfc     GSSLibStub.obj
 0002:00000e24       ??_C@_0BE@LBCEEBKN@?$FLGSSLibStub_unwrap?$FN@ 10006e24     GSSLibStub.obj
 0002:00001070       _JAVA_DUPLICATE_TOKEN_CODE 10007070     NativeUtil.obj
 0002:00001074       _JAVA_OLD_TOKEN_CODE       10007074     NativeUtil.obj
 0002:00001078       _JAVA_UNSEQ_TOKEN_CODE     10007078     NativeUtil.obj
 0002:0000107c       _JAVA_GAP_TOKEN_CODE       1000707c     NativeUtil.obj
 0002:00001080       _JAVA_ERROR_CODE           10007080     NativeUtil.obj
 0002:000010c8       _SPNEGO_BYTES              100070c8     NativeUtil.obj
 0002:000010d0       _JAVA_MAX                  100070d0     NativeUtil.obj
 0002:000010d4       ??_C@_0BB@DDFKOHA@java?1lang?1Object@ 100070d4     NativeUtil.obj
 0002:000010e8       ??_C@_0BM@IGAFBDKG@Couldn?8t?5find?5Object?5class?6@ 100070e8     NativeUtil.obj
 0002:00001104       ??_C@_0BB@FLFAIHG@java?1lang?1String@ 10007104     NativeUtil.obj
 0002:00001118       ??_C@_0BM@LOBNDLCB@Couldn?8t?5find?5String?5class?6@ 10007118     NativeUtil.obj
 0002:00001134       ??_C@_0BC@LECFJELF@org?1ietf?1jgss?1Oid@ 10007134     NativeUtil.obj
 0002:00001148       ??_C@_0CH@PGPGONKK@Couldn?8t?5find?5org?4ietf?4jgss?4Oid@ 10007148     NativeUtil.obj
 0002:00001170       ??_C@_0BL@FNACHLFG@org?1ietf?1jgss?1GSSException@ 10007170     NativeUtil.obj
 0002:0000118c       ??_C@_0DA@GFNNKFCG@Couldn?8t?5find?5org?4ietf?4jgss?4GSS@ 1000718c     NativeUtil.obj
 0002:000011bc       ??_C@_0CJ@MAIAMGJJ@sun?1security?1jgss?1wrapper?1GSSNa@ 100071bc     NativeUtil.obj
 0002:000011e8       ??_C@_0DO@BINJABLK@Couldn?8t?5find?5sun?4security?4jgss@ 100071e8     NativeUtil.obj
 0002:00001228       ??_C@_0CJ@GNJHDBAK@sun?1security?1jgss?1wrapper?1GSSCr@ 10007228     NativeUtil.obj
 0002:00001254       ??_C@_0DO@KDKPMOPA@Couldn?8t?5find?5sun?4security?4jgss@ 10007254     NativeUtil.obj
 0002:00001294       ??_C@_0CL@KFFCDPKJ@sun?1security?1jgss?1wrapper?1Nativ@ 10007294     NativeUtil.obj
 0002:000012c0       ??_C@_0EA@KEIEKLLE@Couldn?8t?5find?5sun?4security?4jgss@ 100072c0     NativeUtil.obj
 0002:00001300       ??_C@_0CM@FIPIMGBP@sun?1security?1jgss?1wrapper?1SunNa@ 10007300     NativeUtil.obj
 0002:00001330       ??_C@_0EB@CKAABFEK@Couldn?8t?5find?5sun?4security?4jgss@ 10007330     NativeUtil.obj
 0002:00001374       ??_C@_05GBDANG@?$CI?$FLB?$CJV@ 10007374     NativeUtil.obj
 0002:0000137c       ??_C@_06FALKBLGB@?$DMinit?$DO@ 1000737c     NativeUtil.obj
 0002:00001384       ??_C@_0CK@EGDHFDIO@Couldn?8t?5find?5String?$CIbyte?$FL?$FN?$CJ?5co@ 10007384     NativeUtil.obj
 0002:000013b0       ??_C@_0CH@EFPONDAE@Couldn?8t?5find?5Oid?$CIbyte?$FL?$FN?$CJ?5const@ 100073b0     NativeUtil.obj
 0002:000013d8       ??_C@_04LHPAGAEF@?$CI?$CJ?$FLB@ 100073d8     NativeUtil.obj
 0002:000013e0       ??_C@_06JCEDDFJL@getDER@   100073e0     NativeUtil.obj
 0002:000013e8       ??_C@_0CD@BPHKINPK@Couldn?8t?5find?5Oid?4getDER?$CI?$CJ?5meth@ 100073e8     NativeUtil.obj
 0002:0000140c       ??_C@_0BK@ECDCMHPE@org?1ietf?1jgss?1MessageProp@ 1000740c     NativeUtil.obj
 0002:00001428       ??_C@_0CP@OAIPCLPB@Couldn?8t?5find?5org?4ietf?4jgss?4Mes@ 10007428     NativeUtil.obj
 0002:00001458       ??_C@_03MMPFGPID@?$CI?$CJZ@ 10007458     NativeUtil.obj
 0002:0000145c       ??_C@_0L@DHFIMONM@getPrivacy@ 1000745c     NativeUtil.obj
 0002:00001468       ??_C@_0CP@ELGGFPHK@Couldn?8t?5find?5MessageProp?4getPr@ 10007468     NativeUtil.obj
 0002:00001498       ??_C@_03KNBKCOBB@?$CI?$CJI@ 10007498     NativeUtil.obj
 0002:0000149c       ??_C@_06MKCFHFGC@getQOP@   1000749c     NativeUtil.obj
 0002:000014a4       ??_C@_0CL@HPEKBOID@Couldn?8t?5find?5MessageProp?4getQO@ 100074a4     NativeUtil.obj
 0002:000014d0       ??_C@_04LHKBAEFM@?$CIZ?$CJV@ 100074d0     NativeUtil.obj
 0002:000014d8       ??_C@_0L@CJHHHJJF@setPrivacy@ 100074d8     NativeUtil.obj
 0002:000014e4       ??_C@_0DG@IIGPDELO@Couldn?8t?5find?5MessageProp?4setPr@ 100074e4     NativeUtil.obj
 0002:0000151c       ??_C@_04PFANPMCN@?$CII?$CJV@ 1000751c     NativeUtil.obj
 0002:00001524       ??_C@_06FJLEMNLP@setQOP@   10007524     NativeUtil.obj
 0002:0000152c       ??_C@_0CO@MPIMJBGL@Couldn?8t?5find?5MessageProp?4setQO@ 1000752c     NativeUtil.obj
 0002:0000155c       ??_C@_0BL@NJFIGAKL@?$CIZZZZILjava?1lang?1String?$DL?$CJV@ 1000755c     NativeUtil.obj
 0002:00001578       ??_C@_0BH@MMNNCMHK@setSupplementaryStates@ 10007578     NativeUtil.obj
 0002:00001590       ??_C@_0DO@DMHBAJGD@Couldn?8t?5find?5MessageProp?4setSu@ 10007590     NativeUtil.obj
 0002:000015d0       ??_C@_0BI@GGPJCDGB@?$CIIILjava?1lang?1String?$DL?$CJV@ 100075d0     NativeUtil.obj
 0002:000015e8       ??_C@_0DK@MKODGPFC@Couldn?8t?5find?5GSSException?$CIint?0@ 100075e8     NativeUtil.obj
 0002:00001624       ??_C@_0BN@PCMKHBAM@org?1ietf?1jgss?1ChannelBinding@ 10007624     NativeUtil.obj
 0002:00001644       ??_C@_0DC@KLFKEJOB@Couldn?8t?5find?5org?4ietf?4jgss?4Cha@ 10007644     NativeUtil.obj
 0002:00001678       ??_C@_0BJ@PCBGABPN@?$CI?$CJLjava?1net?1InetAddress?$DL@ 10007678     NativeUtil.obj
 0002:00001694       ??_C@_0BE@BFCHFIIG@getInitiatorAddress@ 10007694     NativeUtil.obj
 0002:000016a8       ??_C@_0DL@FKEIDKDF@Couldn?8t?5find?5ChannelBinding?4ge@ 100076a8     NativeUtil.obj
 0002:000016e4       ??_C@_0BD@GABBFHOC@getAcceptorAddress@ 100076e4     NativeUtil.obj
 0002:000016f8       ??_C@_0DK@IABBFOKP@Couldn?8t?5find?5ChannelBinding?4ge@ 100076f8     NativeUtil.obj
 0002:00001734       ??_C@_0BD@IGFAEMMP@getApplicationData@ 10007734     NativeUtil.obj
 0002:00001748       ??_C@_0DK@JBGAFLDN@Couldn?8t?5find?5ChannelBinding?4ge@ 10007748     NativeUtil.obj
 0002:00001784       ??_C@_0BF@LNJHKELF@java?1net?1InetAddress@ 10007784     NativeUtil.obj
 0002:0000179c       ??_C@_0CK@FNACPNDF@Couldn?8t?5find?5java?4net?4InetAddr@ 1000779c     NativeUtil.obj
 0002:000017c8       ??_C@_0L@KDPCDPCO@getAddress@ 100077c8     NativeUtil.obj
 0002:000017d4       ??_C@_0CP@HGHKJAFB@Couldn?8t?5find?5InetAddress?4getAd@ 100077d4     NativeUtil.obj
 0002:00001804       ??_C@_0CL@DOONCHMP@?$CIJLsun?1security?1jgss?1wrapper?1GS@ 10007804     NativeUtil.obj
 0002:00001830       ??_C@_0DM@MCLCHDAJ@Couldn?8t?5find?5GSSNameElement?$CIlo@ 10007830     NativeUtil.obj
 0002:00001870       ??_C@_0EC@KINGCJOP@?$CIJLsun?1security?1jgss?1wrapper?1GS@ 10007870     NativeUtil.obj
 0002:000018b4       ??_C@_0DM@LOKCAJBC@Couldn?8t?5find?5GSSCredElement?$CIlo@ 100078b4     NativeUtil.obj
 0002:000018f0       ??_C@_0DO@FNIKKMPE@Couldn?8t?5find?5NativeGSSContext?$CI@ 100078f0     NativeUtil.obj
 0002:00001930       ??_C@_0CF@GLMFJBKG@sun?1security?1jgss?1wrapper?1GSSLi@ 10007930     NativeUtil.obj
 0002:00001958       ??_C@_0DK@DKLJHFGN@Couldn?8t?5find?5sun?4security?4jgss@ 10007958     NativeUtil.obj
 0002:00001994       ??_C@_01LELAEKIP@J@        10007994     NativeUtil.obj
 0002:00001998       ??_C@_05ODBFMIC@pMech@     10007998     NativeUtil.obj
 0002:000019a0       ??_C@_0CG@KDHAILGJ@Couldn?8t?5find?5GSSLibStub?4pMech?5@ 100079a0     NativeUtil.obj
 0002:000019c8       ??_C@_08BAFMHLII@pContext@ 100079c8     NativeUtil.obj
 0002:000019d4       ??_C@_0CP@ENCPPLKK@Couldn?8t?5find?5NativeGSSContext?4@ 100079d4     NativeUtil.obj
 0002:00001a04       ??_C@_0CL@POIDEFHJ@Lsun?1security?1jgss?1wrapper?1GSSN@ 10007a04     NativeUtil.obj
 0002:00001a30       ??_C@_07HBEJLLMM@srcName@  10007a30     NativeUtil.obj
 0002:00001a38       ??_C@_0CO@DONIBCN@Couldn?8t?5find?5NativeGSSContext?4@ 10007a38     NativeUtil.obj
 0002:00001a68       ??_C@_0L@JFDMNPJH@targetName@ 10007a68     NativeUtil.obj
 0002:00001a74       ??_C@_0DB@DDBEJNEH@Couldn?8t?5find?5NativeGSSContext?4@ 10007a74     NativeUtil.obj
 0002:00001aa8       ??_C@_01POHCFINO@Z@        10007aa8     NativeUtil.obj
 0002:00001aac       ??_C@_0M@EGOKMCMC@isInitiator@ 10007aac     NativeUtil.obj
 0002:00001ab8       ??_C@_0DC@LNCJDFLL@Couldn?8t?5find?5NativeGSSContext?4@ 10007ab8     NativeUtil.obj
 0002:00001aec       ??_C@_0O@IOAFJPFC@isEstablished@ 10007aec     NativeUtil.obj
 0002:00001afc       ??_C@_0DE@LNDCMEKK@Couldn?8t?5find?5NativeGSSContext?4@ 10007afc     NativeUtil.obj
 0002:00001b30       ??_C@_0CL@JHCIJAHA@Lsun?1security?1jgss?1wrapper?1GSSC@ 10007b30     NativeUtil.obj
 0002:00001b5c       ??_C@_0O@CPAICCNI@delegatedCred@ 10007b5c     NativeUtil.obj
 0002:00001b6c       ??_C@_0DE@DKEHMLGM@Couldn?8t?5find?5NativeGSSContext?4@ 10007b6c     NativeUtil.obj
 0002:00001ba0       ??_C@_01JPJNBJEM@I@        10007ba0     NativeUtil.obj
 0002:00001ba4       ??_C@_05GECEPKB@flags@     10007ba4     NativeUtil.obj
 0002:00001bac       ??_C@_0CM@DLHPFAAC@Couldn?8t?5find?5NativeGSSContext?4@ 10007bac     NativeUtil.obj
 0002:00001bd8       ??_C@_08MOKDPMFA@lifetime@ 10007bd8     NativeUtil.obj
 0002:00001be4       ??_C@_0CP@NKFJJLMO@Couldn?8t?5find?5NativeGSSContext?4@ 10007be4     NativeUtil.obj
 0002:00001c14       ??_C@_0BE@LEBOECLA@Lorg?1ietf?1jgss?1Oid?$DL@ 10007c14     NativeUtil.obj
 0002:00001c28       ??_C@_0L@GPNEDCNK@actualMech@ 10007c28     NativeUtil.obj
 0002:00001c34       ??_C@_0DB@ENGNPLHP@Couldn?8t?5find?5NativeGSSContext?4@ 10007c34     NativeUtil.obj
 0002:00001c68       ??_C@_0BL@ENCPOIKC@java?1lang?1OutOfMemoryError@ 10007c68     NativeUtil.obj
 0002:00001c84       ??_C@_0CP@KLPLCPB@?$FLGSSLibStub?3?$CFd?$FN?5?$CFs?5Status?5major@ 10007c84     NativeUtil.obj
 0002:00001cb4       ??_C@_0CD@EABHFLMM@?$FLGSSLibStub?3?$CFd?$FN?5c?1r?1s?5?$DN?5?$CFd?1?$CFd?1?$CF@ 10007cb4     NativeUtil.obj
 0002:00001cd8       ??_C@_0CK@DNKNKJGD@A?5required?5input?5parameter?5cann@ 10007cd8     NativeUtil.obj
 0002:00001d04       ??_C@_0CM@BAFDHAPF@A?5required?5output?5parameter?5can@ 10007d04     NativeUtil.obj
 0002:00001d30       ??_C@_0BK@ONEELEFA@A?5parameter?5was?5malformed@ 10007d30     NativeUtil.obj
 0002:00001d4c       __pRawDllMain              10007d4c     MSVCRT:dll_dllmain.obj
 0002:00001d4c       __pDefaultRawDllMain       10007d4c     MSVCRT:dll_dllmain.obj
 0002:00001dd0       __load_config_used         10007dd0     MSVCRT:loadcfg.obj
 0002:00001e70       ___safe_se_handler_table   10007e70     <linker-defined>
 0002:000020f8       ___rtc_iaa                 100080f8     MSVCRT:initsect.obj
 0002:000020fc       ___rtc_izz                 100080fc     MSVCRT:initsect.obj
 0002:00002100       ___rtc_taa                 10008100     MSVCRT:initsect.obj
 0002:00002104       ___rtc_tzz                 10008104     MSVCRT:initsect.obj
 0002:000029b0       __IMPORT_DESCRIPTOR_KERNEL32 100089b0     kernel32:KERNEL32.dll
 0002:000029c4       __IMPORT_DESCRIPTOR_VCRUNTIME140 100089c4     vcruntime:VCRUNTIME140.dll
 0002:000029d8       __IMPORT_DESCRIPTOR_api-ms-win-crt-stdio-l1-1-0 100089d8     ucrt:api-ms-win-crt-stdio-l1-1-0.dll
 0002:000029ec       __IMPORT_DESCRIPTOR_api-ms-win-crt-heap-l1-1-0 100089ec     ucrt:api-ms-win-crt-heap-l1-1-0.dll
 0002:00002a00       __IMPORT_DESCRIPTOR_api-ms-win-crt-runtime-l1-1-0 10008a00     ucrt:api-ms-win-crt-runtime-l1-1-0.dll
 0002:00002a14       __NULL_IMPORT_DESCRIPTOR   10008a14     kernel32:KERNEL32.dll
 0003:00000000       ___security_cookie_complement 10009000     MSVCRT:gs_cookie.obj
 0003:00000004       ___security_cookie         10009004     MSVCRT:gs_cookie.obj
 0003:00000008       ___scrt_native_dllmain_reason 10009008     MSVCRT:utility.obj
 0003:00000010       ___isa_enabled             10009010     MSVCRT:cpu_disp.obj
 0003:00000014       ___scrt_ucrt_dll_is_in_use 10009014     MSVCRT:ucrt_stubs.obj
 0003:00000448       ?__type_info_root_node@@3U__type_info_node@@A 10009448     MSVCRT:tncleanup.obj
 0003:00000450       ?_OptionsStorage@?1??__local_stdio_scanf_options@@9@4_KA 10009450     MSVCRT:default_local_stdio_options.obj
 0003:00000458       ___scrt_current_native_startup_state 10009458     MSVCRT:utility.obj
 0003:0000045c       ___scrt_native_startup_lock 1000945c     MSVCRT:utility.obj
 0003:0000047c       ___scrt_debugger_hook_flag 1000947c     MSVCRT:utility_desktop.obj
 0003:00000480       ___isa_available           10009480     MSVCRT:cpu_disp.obj
 0003:00000484       ___favor                   10009484     MSVCRT:cpu_disp.obj
 0003:00000488       _MID_GSSException_ctor3    10009488     <common>
 0003:0000048c       _MID_Oid_getDER            1000948c     <common>
 0003:00000490       _MID_Oid_ctor1             10009490     <common>
 0003:00000494       _MID_String_ctor           10009494     <common>
 0003:00000498       _CLS_SunNativeProvider     10009498     <common>
 0003:0000049c       _CLS_GSSException          1000949c     <common>
 0003:000004a0       _CLS_Oid                   100094a0     <common>
 0003:000004a4       _CLS_String                100094a4     <common>
 0003:000004a8       _FID_NativeGSSContext_actualMech 100094a8     <common>
 0003:000004ac       _FID_NativeGSSContext_lifetime 100094ac     <common>
 0003:000004b0       _FID_NativeGSSContext_flags 100094b0     <common>
 0003:000004b4       _FID_NativeGSSContext_delegatedCred 100094b4     <common>
 0003:000004b8       _FID_NativeGSSContext_isEstablished 100094b8     <common>
 0003:000004bc       _FID_NativeGSSContext_isInitiator 100094bc     <common>
 0003:000004c0       _FID_NativeGSSContext_targetName 100094c0     <common>
 0003:000004c4       _FID_NativeGSSContext_srcName 100094c4     <common>
 0003:000004c8       _FID_NativeGSSContext_pContext 100094c8     <common>
 0003:000004cc       _FID_GSSLibStub_pMech      100094cc     <common>
 0003:000004d0       _MID_NativeGSSContext_ctor 100094d0     <common>
 0003:000004d4       _MID_GSSCredElement_ctor   100094d4     <common>
 0003:000004d8       _MID_GSSNameElement_ctor   100094d8     <common>
 0003:000004dc       _MID_InetAddress_getAddr   100094dc     <common>
 0003:000004e0       _MID_ChannelBinding_getAppData 100094e0     <common>
 0003:000004e4       _MID_ChannelBinding_getAcceptorAddr 100094e4     <common>
 0003:000004e8       _MID_ChannelBinding_getInitiatorAddr 100094e8     <common>
 0003:000004ec       _MID_MessageProp_setSupplementaryStates 100094ec     <common>
 0003:000004f0       _MID_MessageProp_setQOP    100094f0     <common>
 0003:000004f4       _MID_MessageProp_setPrivacy 100094f4     <common>
 0003:000004f8       _MID_MessageProp_getQOP    100094f8     <common>
 0003:000004fc       _MID_MessageProp_getPrivacy 100094fc     <common>
 0003:00000500       _CLS_NativeGSSContext      10009500     <common>
 0003:00000504       _CLS_GSSCredElement        10009504     <common>
 0003:00000508       _CLS_GSSNameElement        10009508     <common>
 0003:0000050c       _CLS_Object                1000950c     <common>
 0003:00000510       _JGSS_DEBUG                10009510     <common>
 0003:00000514       _ftab                      10009514     <common>
 0003:00000518       ?_OptionsStorage@?1??__local_stdio_printf_options@@9@9 10009518     <common>
 0003:00000520       ___dyn_tls_init_callback   10009520     <common>

 entry point at        0001:000037d0

 Static symbols

 0000:ffff4000       .debug$S                   10000000     kernel32:KERNEL32.dll
 0000:ffff4000       .debug$S                   10000000     kernel32:KERNEL32.dll
 0000:ffff4000       .debug$S                   10000000     kernel32:KERNEL32.dll
 0000:ffff4000       .debug$S                   10000000     kernel32:KERNEL32.dll
 0000:ffff4000       .debug$S                   10000000     kernel32:KERNEL32.dll
 0000:ffff4000       .debug$S                   10000000     kernel32:KERNEL32.dll
 0000:ffff4000       .debug$S                   10000000     kernel32:KERNEL32.dll
 0000:ffff4000       .debug$S                   10000000     kernel32:KERNEL32.dll
 0000:ffff4000       .debug$S                   10000000     kernel32:KERNEL32.dll
 0000:ffff4000       .debug$S                   10000000     kernel32:KERNEL32.dll
 0000:ffff4000       .debug$S                   10000000     kernel32:KERNEL32.dll
 0000:ffff4000       .debug$S                   10000000     kernel32:KERNEL32.dll
 0000:ffff4000       .debug$S                   10000000     kernel32:KERNEL32.dll
 0000:ffff4000       .debug$S                   10000000     kernel32:KERNEL32.dll
 0000:ffff4000       .debug$S                   10000000     kernel32:KERNEL32.dll
 0000:ffff4000       .debug$S                   10000000     kernel32:KERNEL32.dll
 0000:ffff4000       .debug$S                   10000000     kernel32:KERNEL32.dll
 0000:ffff4000       .debug$S                   10000000     kernel32:KERNEL32.dll
 0000:ffff4000       .debug$S                   10000000     kernel32:KERNEL32.dll
 0000:ffff4000       .debug$S                   10000000     vcruntime:VCRUNTIME140.dll
 0000:ffff4000       .debug$S                   10000000     vcruntime:VCRUNTIME140.dll
 0000:ffff4000       .debug$S                   10000000     vcruntime:VCRUNTIME140.dll
 0000:ffff4000       .debug$S                   10000000     vcruntime:VCRUNTIME140.dll
 0000:ffff4000       .debug$S                   10000000     ucrt:api-ms-win-crt-stdio-l1-1-0.dll
 0000:ffff4000       .debug$S                   10000000     ucrt:api-ms-win-crt-stdio-l1-1-0.dll
 0000:ffff4000       .debug$S                   10000000     ucrt:api-ms-win-crt-stdio-l1-1-0.dll
 0000:ffff4000       .debug$S                   10000000     ucrt:api-ms-win-crt-heap-l1-1-0.dll
 0000:ffff4000       .debug$S                   10000000     ucrt:api-ms-win-crt-heap-l1-1-0.dll
 0000:ffff4000       .debug$S                   10000000     ucrt:api-ms-win-crt-runtime-l1-1-0.dll
 0000:ffff4000       .debug$S                   10000000     ucrt:api-ms-win-crt-runtime-l1-1-0.dll
 0000:ffff4000       .debug$S                   10000000     ucrt:api-ms-win-crt-runtime-l1-1-0.dll
 0000:ffff4000       .debug$S                   10000000     ucrt:api-ms-win-crt-runtime-l1-1-0.dll
 0000:ffff4000       .debug$S                   10000000     ucrt:api-ms-win-crt-runtime-l1-1-0.dll
 0000:ffff4000       .debug$S                   10000000     ucrt:api-ms-win-crt-runtime-l1-1-0.dll
 0000:ffff4000       .debug$S                   10000000     ucrt:api-ms-win-crt-runtime-l1-1-0.dll
 0000:ffff4000       .debug$S                   10000000     ucrt:api-ms-win-crt-runtime-l1-1-0.dll
 0000:ffff4000       .debug$S                   10000000     j2gss.exp
 0000:ffff4000       .debug$S                   10000000     ucrt:api-ms-win-crt-runtime-l1-1-0.dll
 0000:ffff4000       .debug$S                   10000000     ucrt:api-ms-win-crt-runtime-l1-1-0.dll
 0000:ffff4000       .debug$S                   10000000     ucrt:api-ms-win-crt-runtime-l1-1-0.dll
 0000:ffff4000       .debug$S                   10000000     ucrt:api-ms-win-crt-runtime-l1-1-0.dll
 0001:000034b0       ?dllmain_crt_dispatch@@YGHQAUHINSTANCE__@@KQAX@Z 100044b0 f   MSVCRT:dll_dllmain.obj
 0001:00003503       ?dllmain_crt_process_attach@@YAHQAUHINSTANCE__@@QAX@Z 10004503 f   MSVCRT:dll_dllmain.obj
 0001:0000360d       ?dllmain_crt_process_detach@@YAH_N@Z 1000460d f   MSVCRT:dll_dllmain.obj
 0001:0000369f       ?dllmain_dispatch@@YAHQAUHINSTANCE__@@KQAX@Z 1000469f f   MSVCRT:dll_dllmain.obj
 0001:000037a5       ?dllmain_raw@@YGHQAUHINSTANCE__@@KQAX@Z 100047a5 f   MSVCRT:dll_dllmain.obj
 0001:00003914       ___get_entropy             10004914 f   MSVCRT:gs_support.obj
 0001:00003a09       ?find_pe_section@@YAPAU_IMAGE_SECTION_HEADER@@QAEI@Z 10004a09 f   MSVCRT:utility.obj
 0001:00003e80       $$000000                   10004e80     MSVCRT:sehprolg4.obj
 0002:00000e38       _RELEASE_NAME              10006e38     NativeFunc.obj
 0002:00000e4c       _IMPORT_NAME               10006e4c     NativeFunc.obj
 0002:00000e5c       _COMPARE_NAME              10006e5c     NativeFunc.obj
 0002:00000e70       _CANONICALIZE_NAME         10006e70     NativeFunc.obj
 0002:00000e88       _EXPORT_NAME               10006e88     NativeFunc.obj
 0002:00000e98       _DISPLAY_NAME              10006e98     NativeFunc.obj
 0002:00000eac       _ACQUIRE_CRED              10006eac     NativeFunc.obj
 0002:00000ec0       _RELEASE_CRED              10006ec0     NativeFunc.obj
 0002:00000ed4       _INQUIRE_CRED              10006ed4     NativeFunc.obj
 0002:00000ee8       _IMPORT_SEC_CONTEXT        10006ee8     NativeFunc.obj
 0002:00000f00       _INIT_SEC_CONTEXT          10006f00     NativeFunc.obj
 0002:00000f18       _ACCEPT_SEC_CONTEXT        10006f18     NativeFunc.obj
 0002:00000f30       _INQUIRE_CONTEXT           10006f30     NativeFunc.obj
 0002:00000f44       _DELETE_SEC_CONTEXT        10006f44     NativeFunc.obj
 0002:00000f5c       _CONTEXT_TIME              10006f5c     NativeFunc.obj
 0002:00000f70       _WRAP_SIZE_LIMIT           10006f70     NativeFunc.obj
 0002:00000f84       _EXPORT_SEC_CONTEXT        10006f84     NativeFunc.obj
 0002:00000f9c       _GET_MIC                   10006f9c     NativeFunc.obj
 0002:00000fa8       _VERIFY_MIC                10006fa8     NativeFunc.obj
 0002:00000fb8       _WRAP                      10006fb8     NativeFunc.obj
 0002:00000fc4       _UNWRAP                    10006fc4     NativeFunc.obj
 0002:00000fd0       _INDICATE_MECHS            10006fd0     NativeFunc.obj
 0002:00000fe4       _INQUIRE_NAMES_FOR_MECH    10006fe4     NativeFunc.obj
 0002:00001000       _ADD_OID_SET_MEMBER        10007000     NativeFunc.obj
 0002:00001018       _DISPLAY_STATUS            10007018     NativeFunc.obj
 0002:0000102c       _CREATE_EMPTY_OID_SET      1000702c     NativeFunc.obj
 0002:00001048       _RELEASE_OID_SET           10007048     NativeFunc.obj
 0002:0000105c       _RELEASE_BUFFER            1000705c     NativeFunc.obj
 0002:00001d50       _GS_ExceptionPointers      10007d50     MSVCRT:gs_report.obj
 0002:00002108       __sehtable$?dllmain_crt_process_attach@@YAHQAUHINSTANCE__@@QAX@Z 10008108     MSVCRT:dll_dllmain.obj
 0002:00002128       __sehtable$?dllmain_crt_process_detach@@YAH_N@Z 10008128     MSVCRT:dll_dllmain.obj
 0002:00002148       __sehtable$?dllmain_dispatch@@YAHQAUHINSTANCE__@@KQAX@Z 10008148     MSVCRT:dll_dllmain.obj
 0002:00002168       __sehtable$___scrt_is_nonwritable_in_current_image 10008168     MSVCRT:utility.obj
 0002:00002190       .edata                     10008190     j2gss.exp
 0002:000021b8       rgpv                       100081b8     j2gss.exp
 0002:00002234       rgszName                   10008234     j2gss.exp
 0002:000022b0       rgwOrd                     100082b0     j2gss.exp
 0002:000022ee       szName                     100082ee     j2gss.exp
 0002:000022f8       $N00001                    100082f8     j2gss.exp
 0002:00002306       $N00002                    10008306     j2gss.exp
 0002:00002316       $N00003                    10008316     j2gss.exp
 0002:00002352       $N00004                    10008352     j2gss.exp
 0002:0000238c       $N00005                    1000838c     j2gss.exp
 0002:000023cb       $N00006                    100083cb     j2gss.exp
 0002:00002405       $N00007                    10008405     j2gss.exp
 0002:00002441       $N00008                    10008441     j2gss.exp
 0002:0000247b       $N00009                    1000847b     j2gss.exp
 0002:000024b7       $N00010                    100084b7     j2gss.exp
 0002:000024f0       $N00011                    100084f0     j2gss.exp
 0002:0000252d       $N00012                    1000852d     j2gss.exp
 0002:0000256a       $N00013                    1000856a     j2gss.exp
 0002:000025a7       $N00014                    100085a7     j2gss.exp
 0002:000025e1       $N00015                    100085e1     j2gss.exp
 0002:0000261b       $N00016                    1000861b     j2gss.exp
 0002:00002656       $N00017                    10008656     j2gss.exp
 0002:0000268f       $N00018                    1000868f     j2gss.exp
 0002:000026c4       $N00019                    100086c4     j2gss.exp
 0002:00002700       $N00020                    10008700     j2gss.exp
 0002:00002739       $N00021                    10008739     j2gss.exp
 0002:00002774       $N00022                    10008774     j2gss.exp
 0002:000027a7       $N00023                    100087a7     j2gss.exp
 0002:000027e1       $N00024                    100087e1     j2gss.exp
 0002:0000281e       $N00025                    1000881e     j2gss.exp
 0002:0000285f       $N00026                    1000885f     j2gss.exp
 0002:00002899       $N00027                    10008899     j2gss.exp
 0002:000028d3       $N00028                    100088d3     j2gss.exp
 0002:00002908       $N00029                    10008908     j2gss.exp
 0002:00002940       $N00030                    10008940     j2gss.exp
 0002:00002973       $N00031                    10008973     j2gss.exp
 0002:00002c3a       .idata$6                   10008c3a     kernel32:KERNEL32.dll
 0002:00002c96       .idata$6                   10008c96     vcruntime:VCRUNTIME140.dll
 0002:00002d96       .idata$6                   10008d96     ucrt:api-ms-win-crt-stdio-l1-1-0.dll
 0002:00002db6       .idata$6                   10008db6     ucrt:api-ms-win-crt-heap-l1-1-0.dll
 0002:00002dd6       .idata$6                   10008dd6     ucrt:api-ms-win-crt-runtime-l1-1-0.dll
 0003:00000018       _tlsCBCl                   10009018     GSSLibStub.obj
 0003:00000020       ?szMsgBuf@?P@??Java_sun_security_jgss_wrapper_GSSLibStub_init@@9@9 10009020     GSSLibStub.obj
 0003:00000120       ?__proc_attached@@3HA      10009120     MSVCRT:dll_dllmain.obj
 0003:00000128       _GS_ExceptionRecord        10009128     MSVCRT:gs_report.obj
 0003:00000178       _GS_ContextRecord          10009178     MSVCRT:gs_report.obj
 0003:00000460       ?is_initialized_as_dll@@3_NA 10009460     MSVCRT:utility.obj
 0003:00000461       ?module_local_atexit_table_initialized@@3_NA 10009461     MSVCRT:utility.obj
 0003:00000464       ?module_local_atexit_table@@3U_onexit_table_t@@A 10009464     MSVCRT:utility.obj
 0003:00000470       ?module_local_at_quick_exit_table@@3U_onexit_table_t@@A 10009470     MSVCRT:utility.obj
 0004:00000060       $R000000                   1000a060     j2gss.dll.res
